:100000000C94F3000C940E010C940E010C940E0150
:100010000C940E010C940E010C94C2150C940E015C
:100020000C940E010C940E010C9444180C940518B9
:100030000C94C1100C940E010C940E010C940E0142
:100040000C940E010C9435040C940E010C94730F57
:100050000C941F0F0C940E010C940E010C940E01C5
:100060000C940E010C940E010C940E010C940E01D4
:100070004570692D4F5344205665722E302E382E10
:10008000322E350000416B7475656C6C65732053BE
:10009000657474696E67000053657474696E6720D7
:1000A000200000486F6568656E73656E736F72201F
:1000B00000004853206D697420536368616C746557
:1000C0007220000048656164696E6720486F6C6447
:1000D0002000004B6F6D706173732000004B6F6DDB
:1000E0007061737320666978200000475053204187
:1000F0006B74697620000041636873656E6B6F7086
:1001000070656C756E67200000447265687261747A
:100110006520626567722E2000004665686C657216
:100120002046433C2D3E4F5344200000556E7465DD
:10013000727370616E6E756E672000004B65696E3C
:10014000652053657474696E672D416E7A656967C1
:1001500065000050432F4254206973742065696E16
:100160006765736368616C746574000055656265EA
:10017000726E65686D65204C65747A746573205382
:10018000657474696E6700004F4E00002D2D2D00C0
:10019000004550492D4D656E750050616C0050430F
:1001A0002F4254004B656E6E756E670052432D42B0
:1001B000657472696562000045786974004F4E008D
:1001C0002D2D0076767D76767A76767E76767776C3
:1001D000767B76767876767C76767976767D7676A8
:1001E0007A76767E760011241FBECFEFD4E0DEBF94
:1001F000CDBF11E0A0E0B1E0EAE8F2E302C0059073
:100200000D92AC37B107D9F713E0ACE7B1E001C00C
:100210001D92AF3FB107E1F70C941B010C94000055
:1002200082E981BB8FE084BBAC9AAD9A8EE28ABB37
:10023000D99ADD9A08951F931092C7011092C301B5
:100240001092C801A0E0B0E00E943119802D9927DA
:1002500080938301A1E0B0E00E943119802D99279D
:1002600080930001A2E0B0E00E943119802D99270F
:1002700080938401A7E1B0E00E943119802D992775
:1002800080939B01A8E1B0E00E943119802D99274D
:100290008093B2010E946C150E9410010E942504F7
:1002A00080918301813019F40E94020F02C00E94E4
:1002B000F30E7894A89A0E94BB030E9496040E94B1
:1002C0009D088091B20185FF02C00E94A6120E9483
:1002D000E5080E949B108091AC01813021F41092BE
:1002E000AC010E94CD1680917E018130B1F4109254
:1002F0007E018091C701882351F480918301882376
:1003000031F480919001813011F40E9410100E940C
:10031000B4100E94B9100E946A138091810181304B
:10032000B9F58091C701882399F5AA9A0E94030E16
:1003300080919B018823A9F40E94FB070E94EB0691
:100340008091B20180FF04C00E9434110E946A09AA
:100350008091B20183FF02C00E9480160E9443096F
:1003600016C080910201823054F00E94A5080E94BC
:1003700034110E946A090E94670A0E944309809111
:100380000201833024F00E94FB070E94EB06AA982A
:1003900080917C018130C1F58091C7018823A1F54E
:1003A00010927C0180919B01882321F080910201B1
:1003B000833014F00E941A0980919801909199015C
:1003C0000196909399018093980180919801909162
:1003D0009901CC9769F480919601909197010196CB
:1003E0009093970180939601109299011092980131
:1003F0000E94C90A0E94DE0C80918901813021F49B
:100400000E947D0B0E941A0D10917D01113009F0A0
:1004100062CF8091C701882309F05DCF10927D01E2
:100420000E94A5088091B801813019F0823059F4FA
:1004300006C00E94650982E08093B80104C00E9452
:100440003E091093B80180919B01813009F043CFA0
:100450008091C701882309F03ECF80919A018130B5
:1004600009F039CF10929A0180910201813071F028
:1004700082301CF4882339F02ECF823081F0833013
:1004800009F029CF17C00E94650925CF0E943E09B7
:1004900064E084E00E9467020E9497041CCF0E94DF
:1004A0003E0964E084E00E9467020E949D080E9469
:1004B000E50811CF0E943E0964E084E00E946702D3
:1004C0000E949D080E94E5080E941A0904CF482F47
:1004D000D99827E030E0DB98000000000000000021
:1004E00081E090E0022E02C0880F991F0A94E2F783
:1004F000842311F0DA9A01C0DA98000000000000AD
:100500000000DB9A00000000000000002150304095
:100510008FEF2F3F3807F9F627E030E0DB98000037
:1005200000000000000081E090E0022E02C0880F71
:10053000991F0A94E2F7862311F0DA9A01C0DA983B
:100540000000000000000000DB9A00000000000036
:100550000000215030408FEF2F3F3807F9F6DB982D
:10056000DA98D99A089564E084E00E9467026CE406
:1005700080E00E94670210927E0180917E018823B4
:10058000E1F36AE08CE60E94670260E085E00E9489
:10059000670208951F93CF93DF9380917C01882396
:1005A000E1F310927C010E944D1010E00DC080918B
:1005B0008101813011F40E94030E80917C01813011
:1005C00019F410927C0111E09091B30180E01123A5
:1005D00009F481E0992311F4882349F7C8E1D0E0B8
:1005E000882309F4B1C08091E3038093B201809124
:1005F000B201DE01082E0E94391945E850E061E0A1
:1006000082E00E942E0D48E950E062E082E00E9404
:100610002E0D43EA50E064E082E00E942E0D42EB92
:1006200050E065E082E00E942E0D44EC50E066E070
:1006300082E00E942E0D43ED50E067E082E00E94D0
:100640002E0D4DED50E068E082E00E942E0D4BEE45
:1006500050E069E082E00E942E0D47EF50E06AE032
:1006600082E00E942E0D4CE251E06BE082E00E949D
:100670002E0D4091B0015091B10162E084E10E94E1
:10068000EF0C8091B20180FF03C048E851E002C046
:100690004CE851E064E084E10E942E0D8091B201AB
:1006A00081FF03C048E851E002C04CE851E065E03A
:1006B00084E10E942E0D8091B20182FF03C048E8C0
:1006C00051E002C04CE851E066E084E10E942E0D4A
:1006D0008091B20183FF03C048E851E002C04CE8BA
:1006E00051E067E084E10E942E0D8091B20184FF09
:1006F00003C048E851E002C04CE851E068E084E102
:100700000E942E0D8091B20185FF03C048E851E0A0
:1007100002C04CE851E069E084E10E942E0D809116
:10072000B20186FF03C048E851E002C04CE851E046
:100730006AE084E10E942E0D4091F30355276BE09F
:1007400084E10E94EF0C13C045E850E062E082E0D3
:100750000E942E0D4AE151E065E082E00E942E0DDC
:10076000DE010E943119802D99278093B201DF911B
:10077000CF911F9108950E94B30210927C01809145
:100780007C018823E1F340E750E062E087E00E94CB
:100790002E0D0E94970410927C0180917C01882389
:1007A000E1F310927C0180917C018823E1F31092A7
:1007B0007C0164E084E00E9467026CE480E00E94B7
:1007C000670280918301882319F40E94CA021AC02B
:1007D0004CE351E062E082E00E942E0D43E551E0DF
:1007E00064E082E00E942E0D4CE651E066E082E07B
:1007F0000E942E0DA8E1B0E00E943119802D9927AA
:100800008093B20180917C018823E1F310927C01F6
:1008100080917C018823E1F310927C0180917C011E
:100820008823E1F310927C0180917C018823E1F31D
:1008300010927C0180917C018823E1F310927C016D
:1008400064E084E00E946702089582E083BF92E43E
:100850009EBD8EE189BF83E087BD86E982BD90930E
:100860008A0080E280937D0008951F920F920FB658
:100870000F9211248F939F93809180018F5F8093BB
:10088000800180918001883439F591E090937F0157
:10089000109280018091F7038F5F8093F70380911E
:1008A000F703843631F41092F70390937C01909310
:1008B0007D018091F703823311F490937D01809143
:1008C000F6038F5F8093F6038091F6038A3021F45C
:1008D0001092F60390937E019F918F910F900FBE1F
:1008E0000F901F901895282F80538A3010F090E0B9
:1008F00005C0203311F49AE001C0982F822F815453
:100900008A3110F4922F9653822F81568A3110F437
:10091000922F9C532D3211F499E403C02E3209F426
:1009200091E4892F992787FD90950895089560E0B7
:1009300085E00E94670263E886E00E94670260E942
:1009400087E00E94670260E085E00E94670264E839
:1009500086E00E94670261E987E00E94670260E02A
:1009600085E00E94670265E886E00E94670262E90E
:1009700087E00E94670260E085E00E94670266E807
:1009800086E00E94670263E987E00E94670260E0F8
:1009900085E00E94670267E886E00E94670264E9DA
:1009A00087E00E94670260E085E00E94670268E8D5
:1009B00086E00E94670265E987E00E94670260E0C6
:1009C00085E00E94670269E886E00E94670266E9A6
:1009D00087E00E94670260E085E00E9467026AE8A3
:1009E00086E00E94670267E987E00E94670260E094
:1009F00085E00E94670261EA86E00E94670268E97A
:100A000087E00E94670260E085E00E94670262EA78
:100A100086E00E94670269E987E00E94670260E061
:100A200085E00E94670263EA86E00E9467026AE945
:100A300087E00E94670260E085E00E94670264EA46
:100A400086E00E9467026BE987E00E94670260E02F
:100A500085E00E94670265EA86E00E9467026CE911
:100A600087E00E94670260E085E00E94670266EA14
:100A700086E00E9467026DE987E00E94670260E0FD
:100A800085E00E94670267EA86E00E9467026EE9DD
:100A900087E00E94670260E085E00E94670268EAE2
:100AA00086E00E9467026FE987E00E94670260E0CB
:100AB00085E00E9467026FEB86E00E94670260EAB1
:100AC00087E00E94670260E085E00E94670260ECB8
:100AD00086E00E94670261EA87E00E94670260E0A8
:100AE00085E00E94670261EC86E00E94670262EA8C
:100AF00087E00E94670260E085E00E94670262EC86
:100B000086E00E94670263EA87E00E94670260E075
:100B100085E00E94670263EC86E00E94670264EA57
:100B200087E00E94670260E085E00E94670264EC53
:100B300086E00E94670265EA87E00E94670260E043
:100B400085E00E94670265EC86E00E94670266EA23
:100B500087E00E94670260E085E00E94670266EC21
:100B600086E00E94670267EA87E00E94670260E011
:100B700085E00E9467026DED86E00E94670268EAE8
:100B800087E00E94670260E085E00E9467026EEDE8
:100B900086E00E94670269EA87E00E94670260E0DF
:100BA00085E00E9467026FED86E00E9467026AEAB4
:100BB00087E00E94670260E085E00E94670260EEC5
:100BC00086E00E9467026BEA87E00E94670260E0AD
:100BD00085E00E94670261EE86E00E9467026CEA8F
:100BE00087E00E94670260E085E00E94670262EE93
:100BF00086E00E9467026DEA87E00E94670260E07B
:100C000085E00E94670263EE86E00E9467026EEA5A
:100C100087E00E94670260E085E00E94670264EE60
:100C200086E00E9467026FEA87E00E94670260E048
:100C300085E00E9467026BEF86E00E94670260EB2E
:100C400087E00E94670260E085E00E9467026CEF27
:100C500086E00E94670261EB87E00E94670260E025
:100C600085E00E9467026DEF86E00E94670262EBFA
:100C700087E00E94670260E085E00E9467026EEFF5
:100C800086E00E94670263EB87E00E94670260E0F3
:100C900085E00E9467026FEF86E00E94670264EBC6
:100CA00087E00E94670261E085E00E94670260E0E1
:100CB00086E00E94670265EB87E00E94670261E0C0
:100CC00085E00E94670261E086E00E94670266EBB1
:100CD00087E00E9467020895FF920F931F93CF93BE
:100CE000DF938C01F62EEC0117C06D2F772785E07E
:100CF0000E9467026C2F86E00E9467028F2D992761
:100D0000FC01EE0FFF1FE80FF91FE15FFE4F60814E
:100D100087E00E9467022196C8010596C817D90787
:100D200020F3E8012A9617C06D2F772785E00E94EF
:100D300067026C2F86E00E9467028F2D9927FC01C5
:100D4000EE0FFF1FE80FF91FE15FFE4F608187E0A4
:100D50000E9467022196C8010F96C817D90720F391
:100D6000DF91CF911F910F91FF9008950F931F93E3
:100D7000CF93DF938C01EC010EC06D2F772785E0B8
:100D80000E9467026C2F86E00E94670260E087E0A5
:100D90000E9467022196C8010596C817D90768F313
:100DA000E8012A960EC06D2F772785E00E94670222
:100DB0006C2F86E00E94670260E087E00E94670275
:100DC0002196C8010F96C817D90768F3DF91CF9114
:100DD0001F910F9108951F93CF93DF938091F90294
:100DE0009091FA0266E170E00E94FC189B012E5F70
:100DF0003F4F37FD1BC0C9016AE070E00E94FC183C
:100E0000182F1695C9016AE070E00E94FC1887E06F
:100E100090E0861B91092EE130E0829FE001839FE4
:100E2000D00D929FD00D1124279616C03095219594
:100E30003F4FC9016AE070E00E94FC18182F169518
:100E40001C5FC9016AE070E00E94FC188EE1689F97
:100E5000E0011124C950DF4F80910B0190910C01EA
:100E6000C817D90739F080910B0190910C010E94AD
:100E7000B60604C08091B601811721F0612FCE0122
:100E80000E946C061093B601D0930C01C0930B0125
:100E9000DF91CF911F910895AF92BF92DF92EF92B1
:100EA000FF920F931F93CF93DF93CDB7DEB72197B8
:100EB0000FB6F894DEBF0FBECDBF8C01D62E5C01FD
:100EC00019826B2D772785E00E9467026A2D86E0E4
:100ED0000E946702ED2CFF24F701E35DFE4F608165
:100EE00087E00E9467028EE190E0A80EB91E99810A
:100EF000925E99839C3329F7F4EBAF2EB12CA00EB0
:100F0000B11E6B2D772785E00E9467026A2D86E06F
:100F10000E946702F701E35DFE4F608187E00E9457
:100F20006702EEE1F0E0AE0EBF1EC801825F9E4F89
:100F3000A816B90631F721960FB6F894DEBF0FBE9A
:100F4000CDBFDF91CF911F910F91FF90EF90DF9078
:100F5000BF90AF900895EF92FF920F931F93CF939E
:100F6000DF93CDB7DEB721970FB6F894DEBF0FBE83
:100F7000CDBF8C017C0119826F2D772785E00E94FF
:100F800067026E2D86E00E94670260E087E00E94A3
:100F900067028EE190E0E80EF91E9981925E9983D6
:100FA0009C3351F784EBE82EF12CE00EF11E6F2DEF
:100FB000772785E00E9467026E2D86E00E94670217
:100FC00060E087E00E946702EEE1F0E0EE0EFF1EB7
:100FD000C801825F9E4FE816F90649F721960FB6C1
:100FE000F894DEBF0FBECDBFDF91CF911F910F915F
:100FF000FF90EF9008951F93CF93DF938091FB02B2
:101000009091FC0266E170E00E94FC189B012A5F4F
:101010003F4F37FD12C0C9016AE070E00E94FC1822
:10102000182F16951C5FC9016AE070E00E94FC1839
:10103000C6E8D0E0C61BD10913C0309521953F4FBB
:10104000C9016AE070E00E94FC18182F1695C901CA
:101050006AE070E00E94FC18C62FDD27C957DF4FF9
:1010600080910D0190910E01C817D90739F0809138
:101070000D0190910E010E94AB0704C08091B70151
:10108000811721F0612FCE010E944C071093B70108
:10109000D0930E01C0930D01DF91CF911F91089560
:1010A00060E085E00E9467026FEC86E00E946702C4
:1010B0006CE887E00E94670261E085E00E946702B9
:1010C0006BE086E00E9467026DE887E00E9467029D
:1010D0000895EF92FF920F931F93CF93DF937A01BE
:1010E0009EE1699FB0011124680F711D8B01020FF1
:1010F000111D1092F803EB0116C06D2F772785E0C4
:101100000E9467026C2F86E00E9467028091F803BC
:10111000F701E80FF11D60818F5F8093F80387E08E
:101120000E9467022196C017D10738F3DF91CF9153
:101130001F910F91FF90EF90089525E046E051E058
:101140006EE081E00E9469080895CF93DF93CDB7E8
:10115000DEB724970FB6F894DEBF0FBECDBF19825D
:101160001A8285E48B831C82F894789430910B0367
:10117000832F6AE00E94DC18282F0E94DC18482F79
:10118000822F0E94DC18292F832F0E94DC189923BC
:1011900019F48AE08C8301C09C83222319F48AE02D
:1011A0008A8301C02A83498324E0AE014F5F5F4FE9
:1011B00061E083E00E94690824960FB6F894DEBFD0
:1011C0000FBECDBFDF91CF910895CF93DF93CDB701
:1011D000DEB724970FB6F894DEBF0FBECDBF80E216
:1011E0008A839BE0998381E38B839C8321E0AE011A
:1011F0004E5F5F4F61E081E00E9469088091890144
:10120000813079F421E0AE014F5F5F4F62E00E94D0
:10121000690822E0AE014D5F5F4F63E081E00E940C
:10122000690824960FB6F894DEBF0FBECDBFDF91DC
:10123000CF910895CF93DF93CDB7DEB725970FB643
:10124000F894DEBF0FBECDBFDE011196EAE3F1E0F8
:1012500085E001900D928150E1F725E0AE014F5FEE
:101260005F4F67E08CE00E94690825960FB6F894FE
:10127000DEBF0FBECDBFDF91CF9108956CE480E05B
:101280000E946702089580910D0390910E03843BA4
:10129000910554F08091F303992720910B0330912D
:1012A0000C038217930744F08091B801882361F4FE
:1012B00081E08093B80108958091B801181614F464
:1012C0000E943E091092B801089562E480E00E94F5
:1012D00067020895EF92FF920F931F93CF93DF93CE
:1012E000CDB7DEB72F970FB6F894DEBF0FBECDBFD8
:1012F00085E0FE01369611928A95E9F78091030305
:10130000909104036EE170E00E94FC18CB018E0105
:10131000055F1F4F019797FF02C080E090E04AE011
:1013200050E0B8010E947718F80101900020E9F719
:101330003197EE2EE01A1092F803FF240AC00E0F28
:101340001F1FEC0FFD1F83850E947304F80180832B
:10135000F394EF2DFF278E2D992787FD90958E0111
:101360000F5F1F4FE817F90754F3F092F80325E0D9
:10137000AE014A5F5F4F69E085E10E9469082E2D4A
:10138000A80169E089E18E190E9469082F960FB6BD
:10139000F894DEBF0FBECDBFDF91CF911F910F91AB
:1013A000FF90EF900895EF92FF920F931F93CF93CA
:1013B000DF93CDB7DEB72E970FB6F894DEBF0FBE22
:1013C000CDBF19821A821B821C828091A401909148
:1013D000A5018E01065F1F4F4AE050E0B8010E9450
:1013E0007718F80101900020E9F73197EE2EE01A06
:1013F0001092F803FF240AC00E0F1F1FEC0FFD1FF1
:1014000082850E947304F8018083F394EF2DFF27F7
:101410008E2D992787FD90958E010B5F1F4FE81742
:10142000F90754F3F092F80324E0AE014F5F5F4FE9
:1014300066E085E10E9469082E2DA80166E089E139
:101440008E190E9469088091A4019091A501181637
:10145000190664F460E085E00E94670262EC86E0B1
:101460000E9467026CE887E00E9467028091A401F5
:101470009091A50197FF0CC060E085E00E94670293
:1014800062EC86E00E9467026DE887E00E946702D6
:101490008091A4019091A501892B61F460E085E021
:1014A0000E94670262EC86E00E94670260E087E0CB
:1014B0000E9467022E960FB6F894DEBF0FBECDBF16
:1014C000DF91CF911F910F91FF90EF900895EF92D0
:1014D000FF920F931F93CF93DF93CDB7DEB72B9778
:1014E0000FB6F894DEBF0FBECDBFDE011196E7E365
:1014F000F1E083E001900D928150E1F78E01085FE9
:101500001F4F4AE050E0B8018091090390910A030F
:101510000E947718F80101900020E9F73197EE2E2C
:10152000E01A1092F803FF240AC00E0F1F1FEC0FE1
:10153000FD1F80850E947304F8018083F394EF2DD2
:10154000FF278E2D992787FD90958E010C5F1F4FE9
:10155000E817F90754F3F092F80323E0AE014F5F68
:101560005F4F6EE08DE00E9469082E2DA8016EE0AD
:1015700080E18E190E9469082B960FB6F894DEBFA1
:101580000FBECDBFDF91CF911F910F91FF90EF90D4
:101590000895EF92FF920F931F93CF93DF93CDB7F0
:1015A000DEB728970FB6F894DEBF0FBECDBF198205
:1015B0008AE08A8380919601909197018E010A5F5B
:1015C0001F4F4AE050E0B8010E947718F8010190DF
:1015D0000020E9F73197EE2EE01A1092F803FF246D
:1015E0000DC08E010D5F1F4F0E0F1F1FEC0FFD1F53
:1015F00086810E947304F8018083F394EF2DFF2706
:101600008E2D992787FD9095E817F90754F3F092EE
:10161000F80380919601909197018E010D5F1F4F05
:101620000A976CF421E0AE014F5F5F4F6EE081E0FE
:101630000E94690821E0A8016EE082E004C022E077
:10164000A8016EE081E00E94690880919801909164
:1016500099018E010A5F1F4F4AE050E0B8010E94D5
:101660007718F80101900020E9F73197EE2EE01A83
:101670001092F803FF240DC08E010D5F1F4F0E0F57
:101680001F1FEC0FFD1F86810E947304F8018083E9
:10169000F394EF2DFF278E2D992787FD9095E8175E
:1016A000F90754F3F092F803809198019091990111
:1016B0008E010D5F1F4F0A976CF421E0AE014E5F63
:1016C0005F4F6EE084E00E94690821E0A8016EE0AF
:1016D00085E004C022E0A8016EE084E00E94690871
:1016E00028960FB6F894DEBF0FBECDBFDF91CF9125
:1016F0001F910F91FF90EF900895CF92DF92EF929C
:10170000FF920F931F93CF93DF93CDB7DEB72B9745
:101710000FB6F894DEBF0FBECDBF80918A019091C5
:101720008B0180918A0190918B018D5A964230F005
:101730008CEA96E290938B0180938A0180918A01D2
:1017400090918B0164E670E00E94E8187093860126
:101750006093850180918A0190918B0164E670E02D
:101760000E94E818909388018093870180918701F7
:10177000909188016AE070E00E94E81870938801F7
:1017800060938701809185019091860125E42983EA
:101790001A821B828E01085F1F4F4AE050E0B80199
:1017A0000E947718F80101900020E9F73197CE2EBA
:1017B000C01A1092F803DD240BC0020F131FE20EB3
:1017C000F31EF70180810E947304F8018083D39493
:1017D0002D2D33278C2D992787FD909548E0E42EF9
:1017E000F12CEC0EFD1E8E010C5F1F4F28173907E0
:1017F00024F3D092F80322E0AE014E5F5F4F62E027
:1018000083E00E9469082C2DA80162E085E08C1914
:101810000E94690880918701909188014AE050E018
:10182000B7010E947718F70101900020E9F731977E
:10183000EE19EE2E1092F803FF240AC00E0F1F1FA0
:10184000EC0FFD1F80850E947304F8018083F394E0
:10185000EF2DFF278E2D992787FD90958E010C5F28
:101860001F4FE817F90754F3F092F80321E0AE0197
:101870004F5F5F4F62E085E00E94690821E0AE01A2
:101880004E5F5F4F62E086E00E94690821E0A80198
:1018900062E086E00E9469082B960FB6F894DEBFDE
:1018A0000FBECDBFDF91CF911F910F91FF90EF90B1
:1018B000DF90CF9008950F931F93CF93DF93CDB711
:1018C000DEB72A970FB6F894DEBF0FBECDBF4AE051
:1018D00050E08E010F5F1F4FB8010E947718F8018A
:1018E00001900020E9F73197E01B1092F80320E007
:1018F000FF27E7FDF09501C02F5F822F99278E17F4
:101900009F07D4F32093F8032A960FB6F894DEBF0E
:101910000FBECDBFDF91CF911F910F9108959F9280
:10192000AF92BF92CF92DF92EF92FF920F931F93ED
:10193000CF93DF93CDB7DEB76E970FB6F894DEBFC7
:101940000FBECDBF982EA62E7A01FA01019000207D
:10195000E9F73197BE2EB41ACC24DD240BC0FF2743
:101960008A010E0F1F1FEE0DFF1D80810E94730460
:10197000F8018083EC2D0894C11CD11C8B2D992774
:101980000196AE014F5F5F4FC816D90641F72B2D68
:101990006A2D892D0E9469086E960FB6F894DEBFF5
:1019A0000FBECDBFDF91CF911F910F91FF90EF90B0
:1019B000DF90CF90BF90AF909F9008958091840169
:1019C000813061F49091D50197FD9F5F959546ED2B
:1019D00051E061E08EE0891B0E948F0C0895EF9228
:1019E000FF920F931F93CF93DF93CDB7DEB764972A
:1019F0000FB6F894DEBF0FBECDBFE82EF62ECA019B
:101A00004AE050E08E010F5F1F4FB8010E94771827
:101A1000A8016F2D8E2D0E948F0C64960FB6F8943E
:101A2000DEBF0FBECDBFDF91CF911F910F91FF9011
:101A3000EF90089560918C0170918D0180918E01DD
:101A400090918F0128E631E040E050E00E940F19AC
:101A5000A90163E083E00E94EF0C0895BF92CF924A
:101A6000DF92EF92FF920F931F93CF93DF93CDB747
:101A7000DEB764970FB6F894DEBF0FBECDBFB82EA9
:101A8000C62E9A01DE01119605C0EA0FFB1F908356
:101A90002F5F3F4F822F841BF9019491E82FFF277E
:101AA000992399F7EA0FFB1F1082FD010190002096
:101AB000E9F73197DE2EDA1AEE24FF2409C08D01F2
:101AC000020F111DF80180810E947304F8018083C8
:101AD0002E2D0894E11CF11C8D2D99270196DE0115
:101AE0001196E816F90659F72D2DAD016C2D8B2DA9
:101AF0000E94690864960FB6F894DEBF0FBECDBF92
:101B0000DF91CF911F910F91FF90EF90DF90CF90D9
:101B1000BF900895EF92FF920F931F93CF93DF939F
:101B200033E0E32EF12CC0E0D0E0A4E6B2E08C91EB
:101B3000FD01218112810381B7016C5F7F4F7B0121
:101B40001496F2E0633D7F0709F456C0422F5527F3
:101B50004D535040E0914301F0914401EC0FFD1FC3
:101B60009927CD97880F991F880F991F9A0168941C
:101B700013F8359527951694E1F7822B932B8083E4
:101B800067327105C9F1212F33272D533040FE01F3
:101B900031968091430190914401E80FF91F4F70F5
:101BA000507084E0440F551F8A95E1F7C90195955F
:101BB000879595958795482B592B408381E06B3706
:101BC0007807D1F0FE013296809143019091440153
:101BD000E80FF91F2370307086E0220F331F8A95BB
:101BE000E1F7802F9927CD97282B392B20836F5C25
:101BF000724011F023969BCFDF91CF911F910F91EF
:101C0000FF90EF900895EF92FF920F931F93CF9361
:101C1000DF9380916302843409F091C033E0E32EB6
:101C2000F12C60E070E0A4E6B2E08C91FD0121812E
:101C300012810381E70124967E01149661347105B7
:101C400009F456C0422F55274D535040E0913F01B3
:101C5000F0914001E60FF71F9927CD97880F991F44
:101C6000880F991F9A01689413F835952795169453
:101C7000E1F7822B932B808360347105C9F1212F0A
:101C800033272D533040FB01319680913F019091D5
:101C90004001E80FF91F4F70507084E0440F551F4A
:101CA0008A95E1F7C9019595879595958795482B74
:101CB000592B4083CB35D105D9F0FB013296809169
:101CC0003F0190914001E80FF91F2370307046E00A
:101CD000220F331F4A95E1F7802F9927CD97282BA4
:101CE000392B20836E33710519F06D5F7F4F9DCFC7
:101CF00080910D0390910E03843B91058CF48091AB
:101D000090018130E1F410929001F8940E94020F4A
:101D1000789480910D0390910E03843B91057CF0A3
:101D200080919001882359F481E080939001F89488
:101D300080918301882311F40E94F30E789480919E
:101D400063028C3459F481E090E09093B101809368
:101D5000B00181E08093B3010E948A0D80916302FB
:101D60008D3459F482E090E09093B1018093B001FA
:101D700081E08093B3010E948A0D809163028E34CA
:101D800059F483E090E09093B1018093B00181E039
:101D90008093B3010E948A0D809163028F3459F4BD
:101DA00084E090E09093B1018093B00181E0809352
:101DB000B3010E948A0D80916302803559F485E059
:101DC00090E09093B1018093B00181E08093B301E2
:101DD0000E948A0D10928101DF91CF911F910F9186
:101DE000FF90EF90089582E289B910BC80B91CBEC3
:101DF00028E92AB996E890BD82EC8BB921B99CBF3D
:101E000082B9089582E289B910BC80B91CBE88E904
:101E10008AB926E820BD92EC9BB980E981B92CBF34
:101E200092B90895159BFECF83B908955D9BFECFAF
:101E30008CB908955D9BFECF8EE38CB908951F92F7
:101E40000F920FB60F9211248F939F93EF93FF93EE
:101E500093B19093FA039D3081F48091B901813060
:101E600061F4AB981092B90180938101E09139033C
:101E7000FF27EF59FD4F90832DC08091B901882332
:101E800019F0813039F514C0933241F48091810109
:101E9000882321F481E08093B901AB9A1092390331
:101EA00080913903E82FFF27EF59FD4F90830CC035
:101EB000E0913903FF27EF59FD4F9083809139035B
:101EC000853930F4809139038F5F8093390302C0E4
:101ED0001092B901FF91EF919F918F910F900FBEDA
:101EE0000F901F9018951F920F920FB60F9211240A
:101EF0002F933F938F939F93AF93BF93EF93FF9352
:101F00002CB12093F90385B398E0892785BB5D9BAD
:101F1000FECF2CB92D3059F08091DA03E82FFF273E
:101F2000E45CFC4F20838F5F8093DA035CC0E09118
:101F3000DA03FF27E45CFC4F20831092AD0110927E
:101F4000AE011092AF018091DA0390E030E007C05B
:101F50002130C9F0213018F02230D1F527C0A32F4D
:101F6000BB27A45CBC4F8C91803211F421E013C0DC
:101F7000E92FFF278C91EE52FC4F80839093AD01A7
:101F80009F5F20E025C0A32FBB27A45CBC4F8C9192
:101F9000803219F422E090E01BC0E92FFF278C91DA
:101FA000E55CFD4F80839093AE0111C0A32FBB274A
:101FB000A45CBC4F8C91803211F423E0ECCFE92F6C
:101FC000FF278C91E45DFD4F80839093AF019F5F6D
:101FD0003F5F8091DA03831708F0BACF81E08093E6
:101FE000AC011092DA03FF91EF91BF91AF919F91F5
:101FF0008F913F912F910F900FBE0F901F901895CA
:10200000662369F020E030E0FC01E20FF11DE08181
:102010005D9BFECFECB92F5F3F4F6217A8F7089585
:10202000CF93DF93CDB7DEB72A970FB6F894DEBF14
:102030000FBECDBF83E289831A8283E68B831C8225
:102040001D8286E890E060E070E10E94FC189C012F
:1020500060E470E00E94FC18635C6E83C90160E478
:1020600070E00E94FC18835C8F838DE08887FE01FE
:1020700031969E01275F3F4F8081159BFECF83B92C
:102080003196E217F307C1F72A960FB6F894DEBF30
:102090000FBECDBFDF91CF910895CF93DF93CDB722
:1020A000DEB72C970FB6F894DEBF0FBECDBF83E22C
:1020B00089831A8281E78B838CE78C838DE68D83FD
:1020C0008DE38E838F8320E030E0FE013196AE01F8
:1020D000485F5F4F8191280F311DE417F507D1F755
:1020E000C90160E070E10E94FC189C0160E470E0AE
:1020F0000E94FC18635C6887C90160E470E00E947C
:10210000FC18835C89878DE08A87FE0131969E01E9
:10211000255F3F4F8081159BFECF83B93196E21733
:10212000F307C1F72C960FB6F894DEBF0FBECDBFF4
:10213000DF91CF9108955D9BFECF8DE68CB95D9BBD
:10214000FECF8FE68CB95D9BFECF89E68CB95D9B97
:10215000FECF8EE68CB95D9BFECF8DE08CB95D9B8A
:10216000FECF8EE38CB9089585B392E0892785BBB5
:10217000089590919301913019F485B3892785BB17
:1021800008951F920F920FB60F9211242F933F9331
:102190005F936F937F938F939F93AF93BF93809140
:1021A000BB019091BC01892B81F484B595B59093C6
:1021B000C2018093C1018EB58F7B8EBD81E090E01E
:1021C0009093BC018093BB0141C084B595B59093B9
:1021D000C0018093BF012EB520642EBD2091C101A6
:1021E0003091C201821B930B1092BC011092BB0173
:1021F000865698406CE271E00E94E8187093BE0128
:102200006093BD0177FF05C01092BE011092BD0121
:1022100009C06730710534F086E090E09093BE010C
:102220008093BD012091BD013091BE0180910201DA
:10223000992787FD90952817390741F026303105F9
:102240002CF42093020181E080939A01BF91AF9119
:102250009F918F917F916F915F913F912F910F90FF
:102260000FBE0F901F901895809103039091040367
:1022700090939D0180939C0180919C0190919D0180
:1022800020919E0130919F01821B930B9093A1019D
:102290008093A00180919C0190919D0190939F015A
:1022A00080939E014091A8015091A9012091A00125
:1022B0003091A101CA01E3E0880F991FEA95E1F787
:1022C000841B950B73E0220F331F7A95E1F7820F81
:1022D000931F68E070E00E94FC187093A90160935E
:1022E000A8012091AA013091AB014091A801509121
:1022F000A901C90163E0880F991F6A95E1F7821B64
:10230000930B840F951F68E070E00E94FC18709397
:10231000AB016093AA018091AA019091AB019093C7
:10232000A5018093A4010E94D3090895BF92CF9282
:10233000DF92EF92FF920F931F93CF93DF93CDB76E
:10234000DEB760970FB6F894DEBF0FBECDBF19821F
:102350001A821B821C828091220290912302909308
:10236000FE038093FD0380912402909125029093B7
:10237000FC038093FB038091FD039091FE038E018B
:10238000055F1F4F4AE050E0B8010E947718F8013E
:1023900001900020E9F73197BE2EB01ACC24DD243D
:1023A0000DC0EC0CFD1CF70180810E9473040C0D24
:1023B0001D1DF80180830894C11CD11C8B2D992709
:1023C00087FD90952BE0E22EF12CEC0EFD1E8E0188
:1023D0000B5F1F4FC816D90624F324E0AE014F5FF0
:1023E0005F4F61E08CE00E9469082B2DA80161E03D
:1023F00080E18B190E9469088091FB039091FC0396
:102400004AE050E0B7010E947718F70101900020E0
:10241000E9F73197DE2EDE18EE24FF240DC0FE0111
:10242000EE0DFF1D83850E9473040E0D1F1DF80124
:1024300080830894E11CF11C8D2D992787FD9095D0
:102440008E010B5F1F4FE816F9064CF324E0AE0136
:102450004F5F5F4F62E08CE00E9469082D2DA8015C
:1024600062E080E18D190E94690860960FB6F894C9
:10247000DEBF0FBECDBFDF91CF911F910F91FF90B7
:10248000EF90DF90CF90BF900895DF92EF92FF9290
:102490000F931F93CF93DF93CDB7DEB72B970FB674
:1024A000F894DEBF0FBECDBFDE011196EBE4F1E084
:1024B00083E001900D928150E1F78E01085F1F4F7C
:1024C000809160024AE050E0B80199270E94771895
:1024D000F80101900020E9F73197DE2ED01AEE24A2
:1024E000FF240DC0FE01EE0DFF1D80850E947304C8
:1024F0000E0D1F1DF80180830894E11CF11C8D2D29
:10250000992787FD90958E010C5F1F4FE816F906FD
:102510004CF323E0AE014F5F5F4F61E088E10E9422
:1025200069082D2DA80161E08BE18D190E946908D1
:102530002B960FB6F894DEBF0FBECDBFDF91CF91C3
:102540001F910F91FF90EF90DF90089522E049E4F2
:1025500051E061E08AE10E94690808956F927F92DC
:102560008F929F92BF92CF92DF92EF92FF920F9342
:102570001F93CF93DF93CDB7DEB764970FB6F89470
:10258000DEBF0FBECDBF19821A821B821C826090F3
:102590005C0270905D0280905E0290905F028E01FE
:1025A000035F1F4F609158027091590280915A0247
:1025B00090915B022AE030E0A8010E949818F8018F
:1025C00001900020E9F73197BE2EB01ACC24DD240B
:1025D0000DC0EC0CFD1CF70180810E9473040C0DF2
:1025E0001D1DF80180830894C11CD11C8B2D9927D7
:1025F00087FD90953DE0E32EF12CEC0EFD1E8E0143
:102600000B5F1F4FC816D90624F324E0AE014F5FBD
:102610005F4F6DE084E10E9469082B2DA8016DE0F9
:1026200088E18B190E9469082AE030E0A701C40103
:10263000B3010E949818F70101900020E9F7319743
:10264000DE2EDE18EE24FF240DC0FE01EE0DFF1D70
:1026500085850E9473040E0D1F1DF8018083089468
:10266000E11CF11C8D2D992787FD90958E010B5F44
:102670001F4FE816F9064CF324E0AE014F5F5F4FA1
:102680006EE084E10E9469082D2DA8016EE088E1CA
:102690008D190E94690864960FB6F894DEBF0FBECC
:1026A000CDBFDF91CF911F910F91FF90EF90DF9001
:1026B000CF90BF909F908F907F906F900895F894E7
:1026C00088E190E028E00FB6F894A89581BD0FBE90
:1026D00021BDFFCF1F939D9900C18091C3018F5FE2
:1026E0008093C30191E09093C5018091C30185302F
:1026F00009F0F7C08091C701882309F06FC090935B
:10270000C7011092C80164E084E00E94670246EDB0
:1027100051E061E083E00E948F0C41E951E063E009
:1027200083E00E942E0D68E084E00E9467024AE97F
:1027300051E065E083E00E942E0D80910001813020
:1027400019F44DEB51E002C040EC51E065E084E14A
:102750000E942E0D60E084E00E9467024EE951E085
:1027600066E083E00E942E0D80918301813019F490
:102770004DEB51E002C040EC51E066E084E10E9484
:102780002E0D44EA51E067E083E00E942E0D809117
:102790008401813019F44DEB51E002C040EC51E06E
:1027A00067E084E10E942E0D4CEA51E068E083E08E
:1027B0000E942E0D80919B01813019F44DEB51E068
:1027C00002C040EC51E068E084E10E942E0D48EB2D
:1027D00051E06BE083E00E942E0D81C01091C80192
:1027E000113001F568E084E00E9467028091830166
:1027F000882329F4109383014DEB51E004C010921B
:10280000830140EC51E066E084E10E942E0D80914E
:102810008301A0E0B0E0082E0E94391960E084E056
:102820000E9467028091C801823009F568E084E067
:102830000E94670280918401882331F481E08093B3
:1028400084014DEB51E004C01092840140EC51E052
:1028500067E084E10E942E0D80918401A2E0B0E047
:10286000082E0E94391960E084E00E94670280917E
:10287000C801833009F568E084E00E946702809116
:102880009B01882331F481E080939B014DEB51E063
:1028900004C010929B0140EC51E068E084E10E948A
:1028A0002E0D80919B01A7E1B0E0082E0E943919FE
:1028B00060E084E00E9467028091C801843089F45E
:1028C0001092C701F89488E190E028E00FB6F894E0
:1028D000A89581BD0FBE21BDFFCF1092C3011092FC
:1028E000C5019C99E9C09091C701913009F0EAC0F7
:1028F0009093C6018091C4018F5F8093C401809141
:10290000C401853009F0DEC01092C4018091C80175
:10291000823009F464C0833030F4882359F0813068
:1029200009F0D0C031C0833009F483C0843009F08D
:10293000C9C09EC09093C8014AE951E065E083E0B8
:102940000E942E0D80910001813019F44DEB51E071
:1029500002C040EC51E065E084E10E942E0D68E089
:1029600084E00E9467024EE951E066E083E00E9445
:102970002E0D80918301813019F44DEB51E002C09E
:1029800040EC51E066E090C082E08093C8014EE9DF
:1029900051E066E083E00E942E0D8091830181303A
:1029A00019F44DEB51E002C040EC51E066E084E1E7
:1029B0000E942E0D68E084E00E94670244EA51E024
:1029C00067E083E00E942E0D80918401813019F42C
:1029D0004DEB51E002C040EC51E067E065C083E0A0
:1029E0008093C80144EA51E067E00E942E0D809177
:1029F0008401813019F44DEB51E002C040EC51E00C
:102A000067E084E10E942E0D68E084E00E94670286
:102A10004CEA51E068E083E00E942E0D80919B011A
:102A2000813019F44DEB51E002C040EC51E068E018
:102A30003BC084E08093C8014CEA51E068E083E049
:102A40000E942E0D80919B01813019F44DEB51E0D5
:102A500002C040EC51E068E084E10E942E0D68E085
:102A600084E00E94670248EB51E06BE083E01DC008
:102A70001092C80148EB51E06BE083E00E942E0DFC
:102A800068E084E00E9467024AE951E065E083E083
:102A90000E942E0D80910001813019F44DEB51E020
:102AA00002C040EC51E065E084E10E942E0D60E040
:102AB00084E00E94670206C01092C4018091C501A3
:102AC0008091C6011F910895813029F4A0E0B0E003
:102AD000062E0E94391908950F931F93CF93DF9309
:102AE000CDB7DEB764970FB6F894DEBF0FBECDBF8B
:102AF00040E050E08E010F5F1F4F842F9927DC01CB
:102B0000AD5FBF4F0E943119202D3327F801E80F28
:102B1000F91F20832223E1F04F5F5F4F2F3F69F7BA
:102B2000108216C0BD016A527E4FAC0FBD1FFD0161
:102B30008181FB0180831182A22FBB272F5F3F4F32
:102B4000842F992787FD9095A817B9075CF30FC0CC
:102B5000DE011196FD0101900020E9F73197EA1B93
:102B6000FB0B4E2FE093D50120E030E0E5CF6496DB
:102B70000FB6F894DEBF0FBECDBFDF91CF911F918E
:102B80000F9108951F920F920FB60F921124EF929A
:102B9000FF920F931F932F933F934F935F936F93E6
:102BA0007F938F939F93AF93BF93EF93FF93809106
:102BB000C901882389F480918000909181009093CD
:102BC000D0018093CF0180918A008F7B80938A000F
:102BD00081E08093C9017FC0809180009091810045
:102BE00090938B0180938A0180918A008064809306
:102BF0008A0010928900109288001092C901809179
:102C00008A0190918B012091CF013091D001821BDC
:102C1000930B90938B0180938A0180918A0190910C
:102C20008B019695879590938B0180938A01809173
:102C30008A0190918B018456904090938B018093F0
:102C40008A0180918A0190918B019C01442755272C
:102C50008091CA019091CB01A091CC01B091CD019E
:102C6000280F391F4A1F5B1F2093CA013093CB01E5
:102C70004093CC015093CD018091CE01843130F14D
:102C80001092CE01E0908C01F0908D0100918E01A8
:102C900010918F01CA01B90124E130E040E050E019
:102CA0000E940F19E20EF31E041F151FE0928C0103
:102CB000F0928D0100938E0110938F011092CA0142
:102CC0001092CB011092CC011092CD018091CE01D7
:102CD0008F5F8093CE01FF91EF91BF91AF919F9154
:102CE0008F917F916F915F914F913F912F911F91A4
:102CF0000F91FF90EF900F900FBE0F901F901895BF
:102D0000CF93DF93CDB7DEB760970FB6F894DEBFF1
:102D10000FBECDBF8091090390910A0390934702A3
:102D20008093460280914602909147026FE070E0E6
:102D30000E94E818AE014B5F5F4FDA01641BCE01C1
:102D40004096E62FEA0FFF27ED53FE4FE491ED93F7
:102D5000A817B907B1F719821A821B821C822BE0CF
:102D60006EE089E00E94690824E0AE014F5F5F4F8A
:102D70006CE08EE00E946908409146025091470243
:102D80006CE08FE00E94EF0C60960FB6F894DEBF07
:102D90000FBECDBFDF91CF910895CF93DF93CDB715
:102DA000DEB7AD970FB6F894DEBF0FBECDBFDE0124
:102DB0001796EEE4F1E087E001900D928150E1F783
:102DC000DE015796E5E5F1E089E001900D92815032
:102DD000E1F7DE019096EEE5F1E08EE001900D92D4
:102DE0008150E1F7DE011196ECE6F1E086E001901A
:102DF0000D928150E1F7DE011E96E2E7F1E089E0F5
:102E000001900D928150E1F78091D2032091D3037C
:102E10006091D4034091D50390E0883609F491E0A5
:102E200080E0253609F481E09823892F992720E056
:102E300030E0403711F421E030E040E050E06C3603
:102E400011F441E050E02423352382239323892B7E
:102E500091F066E070E0CE0107960E94001068E0F5
:102E600070E0CE0147960E9400106DE070E0CE0148
:102E700080960E9400108091D2032091D30360912C
:102E8000D4034091D50390E0833709F491E080E0CA
:102E9000283609F481E09823892F992720E030E033
:102EA000473711F421E030E040E050E06F3611F494
:102EB00041E050E02423352382239323892B41F1E1
:102EC00080913B0290913C028934A1F4943491F4B6
:102ED00065E070E0CE0101960E9400106091D5017E
:102EE000772767FD709586ED91E00E9400108DE0D8
:102EF0000E94160F80913B0290913C02863741F46C
:102F0000953631F468E070E0CE010E960E94001014
:102F10008091D2032091D3034091D40390E0833772
:102F200009F491E080E0253609F481E09823892FA7
:102F3000992720E030E0443711F421E030E082238B
:102F40009323892B81F180913B0290913C0289343B
:102F500051F5943441F540E050E00FC0F901E45DD3
:102F6000FD4F8081D901AD5FBF4F082E0E943919F6
:102F700080812A523E4FF9018083942F8091AF01C6
:102F80004F5F5F4F292F3327981740F3D901AD5F6B
:102F9000BF4F80E0082E0E9439192A523E4FF90196
:102FA00010829093D5018091D2032091D303609138
:102FB000D4034091D50390E0823709F491E080E09A
:102FC000253609F481E09823892F992720E030E005
:102FD000453611F421E030E040E050E0633711F471
:102FE00041E050E02423352382239323892B11F0E1
:102FF0000E945F130E941A0FAD960FB6F894DEBFC1
:103000000FBECDBFDF91CF9108951F920F920FB6E3
:103010000F9211248F939F938091D4018130A1F05E
:10302000813018F0823049F525C08091D2018E316F
:1030300029F41092D20181E08093D4018091D201D1
:103040008F5F8093D20119C09091D301923061F4C7
:103050001092D3018091D101813019F49093D40161
:1030600003C083E08093D4018091D3018F5F80936C
:10307000D30103C083E08093D4019F918F910F907F
:103080000FBE0F901F9018951F920F920FB60F92C0
:1030900011248F938091D401833011F41092D401C4
:1030A0008F910F900FBE0F901F9018958091F9028D
:1030B0009091FA0265E070E00E94FC1866507F4F24
:1030C00077FD0FC081E0653F78071CF064EF71E089
:1030D00003C06B3F71053CF06A5F81E08093D101D2
:1030E00004C060E070E01092D10162BD0895FB0160
:1030F0009F01E8944230C4F04532B4F44A3029F4D8
:1031000097FB1EF4909581959F4F642F77270E941F
:10311000E818805D8A330CF0895D8193CB010097BC
:10312000A1F716F45DE251931082C9010C94CC18FA
:10313000FA01CF93FF93EF93223044F1253234F517
:10314000C22FE894CA3049F497FB3EF490958095DD
:10315000709561957F4F8F4F9F4F2C2F33274427BA
:103160005527FF93EF930E940F19EF91FF91605D38
:103170006A330CF0695D6193B901CA016050704017
:103180008040904051F716F4CDE2C19310828F91A8
:103190009F91CF910C94CC18DC01FC010190002090
:1031A000E9F73297AE17BF0730F47C9160817083E6
:1031B00031976D93F7CF0895991B79E004C0991F5B
:1031C000961708F0961B881F7A95C9F78095089581
:1031D000AA1BBB1B51E107C0AA1FBB1FA617B7073D
:1031E00010F0A61BB70B881F991F5A95A9F7809559
:1031F0009095BC01CD01089597FB092E07260AD0B2
:1032000077FD04D0E5DF06D000201AF470956195B3
:103210007F4F0895F6F7909581959F4F0895A1E20D
:103220001A2EAA1BBB1BFD010DC0AA1FBB1FEE1F40
:10323000FF1FA217B307E407F50720F0A21BB30B8B
:10324000E40BF50B661F771F881F991F1A9469F707
:1032500060957095809590959B01AC01BD01CF0163
:103260000895E199FECFBFBBAEBBE09A11960DB2B7
:103270000895E199FECFBFBBAEBB0DBA11960FB654
:0A328000F894E29AE19A0FBE089557
:10328A0001010300000A0000440000230023005447
:10329A006466536365526200516100506000506079
:1032AA00005161005262005363655464666768693D
:1032BA006A6B6B6A6968670000005353635353F77C
:1032CA0002EA01DB0348020D0A0A1D0000006865D4
:1032DA006C70200D0073686F772049440D00736885
:1032EA006F772076657273696F6E0D004944203DD1
:0C32FA002000302E382E322E350D000042
:00000001FF
